:020000040800F2
:100000000005002011020008891100088D11000868
:10001000E11100088D110008B51100081302000855
:10002000130200081302000813020008C934000874
:10003000130200081302000813020008130200084C
:10004000130200081302000813020008130200083C
:100050001302000813020008B5390008E13900084E
:100060000D3A0008393A0008653A00081302000802
:10007000130200081302000813020008130200080C
:1000800013020008130200081302000819230008D5
:1000900089230008E923000849240008913A000850
:1000A00013020008130200081302000813020008DC
:1000B000C5370008130200081302000813020008E5
:1000C00013020008130200081302000813020008BC
:1000D0001302000821280008352800081302000830
:1000E000F93A00081302000813020008130200087E
:1000F000130200081302000813020008130200088C
:10010000130200081302000813020008130200087B
:10011000130200081302000813020008130200086B
:10012000130200081302000813020008130200085B
:10013000130200081302000813020008130200084B
:10014000130200081302000813020008130200083B
:10015000130200081302000813020008130200082B
:10016000130200081302000813020008130200081B
:10017000130200081302000813020008130200080B
:1001800013020008130200081302000813020008FB
:1001900013020008130200081302000813020008EB
:1001A00013020008130200081302000813020008DB
:1001B00013020008130200081302000813020008CB
:1001C00013020008130200081302000813020008BB
:1001D00013020008130200081302000813020008AB
:1001E000D0400B1CD1409C46203AD3401843524289
:1001F00063469340184370479140031C90409C46CF
:10020000203A9340194352426346D3401943704702
:1002100002E000F000F8FEE772B6394880F3088883
:10022000384880F3098838484EF60851CEF200016C
:10023000086040F20000CCF200004EF63471CEF2BD
:1002400000010860BFF34F8FBFF36F8F40F20000D3
:10025000C0F2F0004EF68851CEF200010860BFF304
:100260004F8FBFF36F8F4FF00000E1EE100A4EF694
:100270003C71CEF200010860062080F31488BFF3C1
:100280006F8F03F05FF903F03DFA4FF055301F49CF
:100290001B4A91423CBF41F8040BFAE71C49194A3A
:1002A00091423CBF41F8040BFAE71A491A4A1B4B2A
:1002B0009A423EBF51F8040B42F8040BF8E70020C5
:1002C0001749184A91423CBF41F8040BFAE703F082
:1002D0003DF903F06BFA144C144DAC4203DA54F8B8
:1002E000041B8847F9E700F03FF8114C114DAC4270
:1002F00003DA54F8041B8847F9E703F025B9000036
:10030000000500200025002000000008000100205A
:100310000005002088430008002500207C250020DF
:1003200080250020DC420020E0010008E0010008F8
:10033000E0010008E00100082DE9F04F2DED108AE2
:10034000C1F80CD0C3689D46BDEC108ABDE8F08FA3
:10035000002383F311882846A047002002F0E6FD21
:1003600002F08CFD00DFFEE7384B6FF016022DE93E
:10037000F0411A70032200245A7007229C70DC702E
:100380001C715C719C71DC711C725C729A72DC7203
:1003900003F044F8074603F091F80546002839D1E8
:1003A0002B4B9F4238D001339F4238D0294B27F046
:1003B000FF029A4237D1F8B200F052FAA84642F250
:1003C000107400F091FC00F051FA064678B384BB3B
:1003D000464635B1204B9F4203D003F067F8002416
:1003E0002646002003F024F81C4B1B691B0723D46E
:1003F0000EB100F035F800F099FC00F04BFE00F073
:1004000003FF0546D4B900F0F3FC4FF47A7002F014
:1004100093FDF7E78046D4E780460446D1E70446DB
:100420004FF00108CDE780464FF47A74C9E70446DF
:10043000CFE74FF47A74CCE70024DCE700F0E4FE69
:10044000401BA042DFD900F00BF8D8E78025002040
:10045000010007B0000008B0263A09B000040240CD
:1004600010B51E4B1E4953F8042F013200D110BDA8
:100470008B42F8D11B4C1C4B22689A422CD91B4B47
:100480009B6803F1006303F580339A4224D202F0A3
:10049000E1FF02F0F3FF002000F016FE144B0220F3
:1004A000187000F045FE134B1A6C00221A64196E86
:1004B0001A66196E596C5A64596E5A665B6E72B63A
:1004C0000D4A0E4B13601B682268202181F31188AE
:1004D0009D4683F30888104710BD00BFFCFF00084D
:1004E0001C00010804000108FFFF0008802500200F
:1004F0008C2500200038024008ED00E000000108D3
:1005000009490B6849F269009AB21B0C00FB0233DF
:10051000064A0B60136844F2506198B21B0C01FB51
:100520000030106080B27047142500201025002094
:1005300010B500211022044600F016FE034B03CB39
:10054000206061601868A06010BD00BF107AFF1FB6
:10055000F0B51F4CBBB000F057FEA368C31AF92BCF
:1005600030D906AD2346A06028220021284601F09C
:10057000D9FB04F10E0000F0EFFD0023C6B2591DB7
:100580005F1CDBB2B3424FEAC10107DA0E332344EA
:100590000822284601F0C6FB3B46F0E701230393FF
:1005A0000823207B02930B4B0193C1F3CF0130232F
:1005B000059100930146049503A3D3E9002306485F
:1005C00001F080F93BB0F0BD78F6339F93CACD8D32
:1005D000C8350020D5350020A435002070B50D4663
:1005E00014461E4601F014F950B9022E0ED1012C0A
:1005F0000CD112A3D3E90023C5E90023012070BD6B
:10060000052C14D003D8012C09D0002070BD282C53
:1006100009D0302CF9D10BA3D3E90023ECE70BA3CD
:10062000D3E90023E8E70BA3D3E90023E4E70BA316
:10063000D3E90023E0E700BFAFF30080401DA12015
:1006400026812A0B78F6339F93CACD8D9E6AC421EA
:10065000818A46EE26417272DF25D7B7F017304AFD
:1006600039059E5638B504460D46034620222846D5
:10067000002101F057FB22792346032A28BF0322D9
:1006800003F8042F28460222202101F04BFB627957
:100690002346072A28BF072203F8052F28460322EE
:1006A000222101F03FFBA2792346072A28BF072217
:1006B00003F8062F28460322252101F033FB2846A4
:1006C00004F108031022282101F02CFB382038BD4A
:1006D0002DE9F04FFFB01FAE0CAD40F2791280460D
:1006E0000F463046002100F03FFD482200212846F9
:1006F00000F03AFD00F088FD574B4FF47A72B0FBE2
:10070000F2F0186093E80700012385E807002B74D6
:100710000DF1520000236B74FFF70AFF032385F8E5
:100720002030E92385F8213006AB18464B4903F009
:1007300099FA162228643146284685F83C20FFF7AE
:1007400091FF10AB044601460822304601F0EAFA58
:100750000822A1180DF14103304601F0E3FA0DF132
:100760004203082204F11001304601F0DBFA11AB1C
:10077000202204F11801304601F0D4FA12AB4022D5
:1007800004F13801304601F0CDFA14AB082204F12F
:100790007801304601F0C6FA0DF15103082204F148
:1007A0008001304601F0BEFA04F1880A0DF15209C9
:1007B00004F5847B4B465146082230460AF1080A6C
:1007C00001F0B0FAD34509F10109F3D119AB0822C0
:1007D0005946304601F0A6FA04F588744FF0000936
:1007E00095F834304B4510D84FF0000995F83C305F
:1007F0004B4515D92B6C21464B440822304601F05D
:1008000091FA083409F10109F0E7AB6B21464B443A
:100810000822304601F086FA083409F10109DFE7C1
:10082000E31DC3F3CF03F97E0593002304960393DE
:10083000BB7E0293193701230093019704A3D3E9E8
:100840000023404601F03EF87FB0BDE8F08F00BFC6
:100850009E6AC421818A46EE902500201C3E000835
:10086000014B1870704700BF04250020F0B52E4BD7
:100870001C7B85B02CB12D4B0E221A81002005B0B7
:10088000F0BD2B4A1068516802AB03C308230DEB7F
:1008900003022849284803F0C7F9054630B9234B1D
:1008A00026480A221A8100F067FCE7E70369B3F5DE
:1008B000E02F07D91D4A22480B211181194600F06B
:1008C0005BFCDBE7418B40F2E932914206D0174BEB
:1008D0000C2018811B4800F04FFCCFE71A4A16493C
:1008E0000244103B20469E1A00F092FC3246074616
:1008F00005F11801204600F08BFCAB689F4202D145
:10090000EB6898420AD0094B0D221A8100903B46B1
:10091000EA68A9680D4800F02FFCAFE70C4800F02A
:100920002BFC0120ABE700BFC8350020902500203C
:100930000C3D0008DCFF060000000108143D000823
:10094000203D0008323D00080800FFF7503D000838
:10095000793D00082DE9F04FAFB006AF80460D4657
:1009600000F056FF0446002875D12B7E022B21D1C2
:10097000EB8A012B1ED100F047FC8146FFF7C0FD3A
:1009800007EE900A9FEDA97AA94EF8EE676A09F57D
:100990001670C6EE877A9FEDA77A67EE877AFCEE2F
:1009A000E77A17EE903A03443360EB7E93B9A24B9B
:1009B00000221A70A437BD46BDE8F08F07F10C0382
:1009C0001C440094002308224FEAC901284601F084
:1009D0000DF84C46AB8A013BA3425FFA84F90BD970
:1009E00004F10109B9F1110FE8D1944B944A40F296
:1009F0003911944803F0EAF807F11C00FFF798FD5D
:100A0000224607F11C0107F10C0003F0FDF8034634
:100A10000028CCD1B9F1100F07D0874B83F8009094
:100A20003368A3F516733360C4E707F1A0020146EB
:100A300002F8950D28460092072200F0D7FFF97AB8
:100A40007F2904DD804B7E4A4FF4A871D1E74046F0
:100A500000F0C2FEAEE7EB8A052B00F02F8106D82E
:100A6000012BA7D129464046FFF732FEA2E7282BEB
:100A70003DD0302B9ED16B7E744C0133627BDBB258
:100A80009342EA4640F01881EA7E237B9A4240F086
:100A9000138107F1A003002623F8846D1022009330
:100AA00031460123284600F0A1FFB5F81480A8F1D3
:100AB00002081FFA88F808F1030323F003030A333E
:100AC00023F00703ADEB030D0DF1180933469BB27C
:100AD000B11C98454FEAC10106F101066DDD4B449A
:100AE000009308220023284600F080FFEEE7AB8A3F
:100AF000013B9BB2C92B3FF65DAF544E347B4CBBE0
:100B000006F10C030093082223462146284600F0F4
:100B10006DFFAB8A04F10109013BE4B29C424FEA4C
:100B2000C90109DA0E34344400940023082228460F
:100B300000F05CFF4C46ECE700230022C6E90023EE
:100B40000023B36086F8D730C6F8D830337B0BB9B2
:100B5000EB7E3373002407F11C0607F10C03082217
:100B600021463046FC603C617C6101F0DBF83B7C57
:100B700004F10109A3424FEAC90107D97B690822A0
:100B80002344304601F0CEF84C46F0E7C1F3CF01E4
:100B90000023E87E059104960393AB7E02931935FA
:100BA00028230146009301951EA3D3E90023404664
:100BB00000F088FEFFF7CCFCFCE694F8D70000F0CC
:100BC00095FAD4F8D83006461BB994F8D70000F04F
:100BD0009DFAD4F8D83043449E4204D294F8D7000A
:100BE000013000F093FA1A4B4FEA980B0025AAB295
:100BF0005A4510462EDA5AB994F8D72042B9D4E9AA
:100C000000120A4304D1D9F800201A600135EEE73A
:100C1000226859F820107B6002EB800000F056FA41
:100C20007B68F3E726417272DF25D7B700FF7F4765
:100C3000A03500200000C8439D350020883D0008F5
:100C4000343E0008E13D0008033E0008C83500209E
:100C500000250020D4E90023D4F8D85012EB080076
:100C600043F10001C4E90001454494F8D700C4F8F9
:100C7000D85000F03BFA854209D394F8D7300133BD
:100C800084F8D730D4F8D8309E1BC4F8D860B8F1B7
:100C9000FF0F0ADC104B00201968207300F016FAD1
:100CA000FFF7E4FD08B1FFF7DBFB23680B4A9B0A63
:100CB000013313810023A360D5467BE6BFF34F8F3A
:100CC0000749084BCA6802F4E0621343CB60BFF3E4
:100CD0004F8F00BFFDE700BF0025002090250020BA
:100CE00000ED00E00400FA0508B54FF000530B4A90
:100CF000196891420AD10A4A597D117009481B7D31
:100D00000373C92208490E3000F01CFAE0220021CA
:100D10004FF00050BDE8084000F026BA9AAD44C537
:100D200004250020C83500201600002030B5254CD1
:100D30002549264885B00223637100250123062238
:100D4000ADF80C508DF80B308DF80C304FF00513CA
:100D50004B60ADF808208DF80A2001F0C9FD1C4B4E
:100D600000931C491C4B01954FF480521B4800F026
:100D7000FDFC1B4B197811B1184800F02DFD00F057
:100D800043FA0546FFF7BCFB07EE900A9FED157A84
:100D9000F8EE676A05F51670C6EE877A9FED127A4F
:100DA00067EE877AFCEEE77A17EE903A034418462E
:100DB0000E4B186002F082FB08B10F23238105B0AF
:100DC00030BD00BF9025002008250020B836002047
:100DD000DD0500089C25002055090008A4350020E9
:100DE0000425002000FF7F470000C843A0350020F5
:100DF0002DE9F04F9DA7D7E900670FF27829D9E9CF
:100E00000089934C93B0DFF874B2DFF874A22046E7
:100E100000F0A4FD0CAD079098B3102200212846E5
:100E200000F0A2F9079B197B4FF0000261F3030267
:100E300019468DF8302051F8040F49680EAA03C2F4
:100E40001B680D9A63F31C029DF830300D9243F03D
:100E500020038DF8303000232A461946584601F009
:100E600057FD079030B9204600F07CFD079B8AF8BB
:100E70000030CCE79AF80030072B40DC01338AF8C9
:100E8000003018220021284600F06EF9DFF8ECB19E
:100E9000DFF8F0A1002319462A46584601F060FD0C
:100EA000014680BB102208A800F05EF9DAF8143081
:100EB00083F48053CAF8143000F0A8F90B4612A945
:100EC000024611E903000DF1240E8EE803009DF89F
:100ED0003410C1F3030089064CBF0E99BDF83810D9
:100EE0008DF82C0046BFC1F31C0141F00041C1F355
:100EF0000A010891204608A900F07AFFCAE72046B7
:100F000000F030FDBDE7204600F082FC824600285C
:100F100052D100F079F94F4B1A6890424CD30793A5
:100F200000F072F98346FFF7EBFA07EE900A9FEDA7
:100F30004A7A8DF820A0F8EE676A0BF51670C6EEB7
:100F4000877ADFF844B19BF800109FED447A67EE92
:100F5000877AFCEEE77A17EE903A03441846079B2F
:100F6000186011B901238DF8203028460791FFF74A
:100F7000DFFA0799C1F1100A5FFA8AFABAF1060F8F
:100F800028BF4FF0060A524629440DF1210000F017
:100F9000D9F80AF10103049308AB039318230293D1
:100FA0002F4B01930123009332463B46204600F02D
:100FB00031FC00238BF8003000F026F9294ADFF8D5
:100FC000CCA01368C31AB3F57A7F32D3106000F057
:100FD0001DF902460B46204600F0CAFC204600F0F0
:100FE00017FC30B39AF80C30DFF8A4B0002B14BF14
:100FF000032302238BF8053000F006F94FF47A73CF
:101000002946B0FBF3F0CBF800005846FFF72AFB67
:10101000182307300293144B0193C0F3CF0040F222
:10102000551304900093039542464B46204600F02A
:10103000F1FB9AF80C300BB1FFF78AFA9AF80C30F2
:10104000002B7FF4E0AE13B0BDE8F08FAFF300806B
:10105000A4350020A035002000FF7F470000C843D2
:101060009C350020A8360020AC360020401DA12071
:1010700026812A0BF1C6A7C1D068080FB836002018
:10108000AD360020000402409D350020C835002008
:101090009025002070B502F079F8094C094E2070B7
:1010A000002530682378834208D902F069F8336854
:1010B00005440133B5F5803F3360F2D370BD00BF06
:1010C000B4360020B036002002F010B907B502ABEC
:1010D00000F1006043F8041D0422194600F5803039
:1010E00002F09AF803B05DF804FB0000054B1A68A3
:1010F000054B1B789B1A834202D9104402F040B87A
:1011000000207047B0360020B436002038B5074DB7
:1011100004462868204402F03BF828B92868204497
:10112000BDE8384002F04CB838BD00BFB0360020F2
:10113000022802BF024B4FF080529A61704700BFF5
:101140000004024010B50023934203D0CC5CC45489
:101150000133F9E710BD000002460346981A13F95F
:10116000011B0029FAD1704702440346934202D082
:1011700003F8011BFAE770470FB4002004B0704772
:101180000EB4002003B07047FEE7000000B59BB02E
:10119000EFF3098168226846FFF7D4FFEFF3058378
:1011A000034B9A6B9A6A9A6A9A6A9A6A9B6AFEE7F2
:1011B00000ED00E000B59BB0EFF3098168226846BE
:1011C000FFF7C0FFEFF30583044B9A6B9A6A9A6AA4
:1011D0009A6A9A6A9A6A9B6AFEE700BF00ED00E08D
:1011E00000B59BB0EFF3098168226846FFF7AAFFBC
:1011F000EFF30583034B5A6B9A6A9A6A9A6A9A6A62
:101200009B6AFEE700ED00E002F0BAB802F0A4B875
:1012100030B5084D0A4491420BD011F8013B092426
:101220005840013CF7D040F300032B4083EA5000C4
:10123000F7E730BD2083B8ED0246006848B1036887
:101240001360D388118901339BB29942D38038BF90
:101250001381704770B588B00D46044620220021E6
:101260006846FFF781FF20460495FFF7E5FF054636
:1012700058B16B46044608AE1A4603CAB242206013
:101280006160134604F10804F6D1284608B070BD29
:101290002DE9F04130B9274B274A40F2C5312748A4
:1012A00002F094FC0B7C23B9254B234A40F2C63153
:1012B000F5E7C66986B9C161BDE8F081002B29DA7E
:1012C000930CAB4229D1B44201D10C60F3E7C8F8CA
:1012D00000100C60BDE8F0814B6823F06047BD0C46
:1012E0004FEAD37EC3F3807C15EA230538BF3D4621
:1012F000B04634466368BEEBD37F23F06042DDD155
:10130000974203D1C3F380739C450AD1974205E00D
:101310001C46EFE7AA4206D013469D422CBF00238D
:101320000123002BCFD12368A046002BF0D12160F0
:10133000BDE8F08108410008FC3E0008C0410008FB
:10134000E141000808B5034A034B044840F25E310E
:1013500002F03CFCD83E000880410008C041000873
:1013600008B503680B60C388016033B9044B054AB4
:1013700005484FF4C76102F029FC013BC38008BD5A
:10138000504100084C3F0008C041000870B50C46B1
:1013900000F10C05616831B9E38A61F30903E38266
:1013A0000020002170BD0E682846FFF7D9FF666057
:1013B000F0E7000008B5426832B10B4B0B4A0C480D
:1013C00040F22F4102F002FCC37DC3F384010131DE
:1013D00061F38603C375C38A62F30903C3821B0AE0
:1013E00062F3C713C37508BD9C410008083F00089D
:1013F000C04100082DE9F047089E32B91F4B204A32
:10140000204840F2395102F0E1FB01F007054FEAB4
:10141000D6082A4406F0070600EBD1004FF47F49B6
:10142000954201D1BDE8F08705F0070E06F0070AE6
:10143000D645774638BF5746C7F10807511BEC0819
:101440008F4228BF0F46045D08EBD60104FA0EF464
:1014500013F801C029FA07FE24FA0AF45FFA8EFE97
:101460008CEA04044EFA0AFE04EA0E048CEA040C28
:1014700003F801C03D443E44D2E700BF1C410008D0
:10148000203F0008C04100082DE9F04106460F4604
:1014900000254FF6FF7441F221082A4630463946AE
:1014A000FEF79EFEC0B284EA0024082314F4004F25
:1014B0004FEA4404A4B203F1FF3318BF84EA0804DE
:1014C00013F0FF03F2D10835402DE6D12046BDE8E8
:1014D000F081000010B50A4441F22104914200D18C
:1014E00010BD11F8013B80EA0320082310F4004FDF
:1014F0004FEA400080B203F1FF3318BF604013F0A1
:10150000FF03F3D1EAE700002DE9F04F85B08A46EA
:101510008DE80C00BDF83C40814630B9494B4A4A41
:1015200040F26E31494802F051FB11F0604F04D097
:10153000474B454A40F26F31F4E7009B002B7ED0C9
:1015400024B10E9B002B7AD0072C28D809F10C006F
:10155000FFF772FE054628B96FF00205284605B070
:10156000BDE8F08F14220021FFF7FEFD22460E9900
:1015700005F10800FFF7E6FD631C2B74009B1B7848
:101580002C4403F01F0363F03F0323724AF000432F
:101590006B6029464846FFF77BFE0125DEE7019B8D
:1015A0001B0A4FF00008029300F10C034FF0800B70
:1015B0004646454603930398FFF73EFE074600283C
:1015C000CAD014220021FFF7CFFDB6BB9DF804302E
:1015D0003B729DF808307B7202220E9B711E1944EB
:1015E000B4420AD9B8180132D2B211F801EF80F82A
:1015F00008E00136072AB6B2F2D1009B197801F053
:101600001F01B44208BF4FF0400BB81841EA48111F
:101610004BEA0103037201324AF000437B603A74E3
:1016200039464846FFF734FE0135B4422DB288F002
:1016300001084FF0000BBED190E70022CDE76FF01C
:1016400001058BE708410008EC3E0008C041000896
:101650002C4100082DE9F0471E46CB8A9146C3F382
:101660000902062A80460F4619D013460021B0B25F
:101670008DB25A1992B2052A09D9A84210D8FA8A0D
:10168000034463F30902FA820120BDE8F087A8420F
:10169000F3D93A4419F8014094760131E8E700257E
:1016A000FB8A7C68C3F30900821F1C23B2FBF3FA98
:1016B00003FB1A2A1FFA8AF27CB301212368002B4C
:1016C00039D1B31F03441C20B3FBF0F301339BB2A9
:1016D00099420CD2BAF1000F09D14046FFF7ACFD98
:1016E00008B1C0F800A0206008B304460022B6B2DA
:1016F0004FF0000AB54230D2691E49441346E01843
:1017000001339BB211F801EF80F804E001351C2B86
:10171000ADB214D0AE42F2D8ECE74046FFF78CFDF4
:10172000044608B1002303607C60002CDED16FF01A
:101730000200BDE8F087013189B21C46BEE7AE4227
:10174000D8D94046FFF778FD08B1C0F800A0206066
:101750000028ECD004460022CCE7FB8AC3F3090240
:10176000164466F30903FB828EE70000F8B50E46C7
:1017700015461F46044628B9144B154A15484F21F3
:1017800002F024FA24220021FFF7EEFC069B63609E
:10179000079B23626A094FF6FF739A424FF00000DD
:1017A00028BF1A46A7602070A061E06197B204F1DB
:1017B0000C05824205D100232B6027826382A3821D
:1017C000F8BD2E60013035462036F2E704410008AE
:1017D000783E0008C041000808B528B9084B094AFE
:1017E0007321094802F0F2F9037823B94BB2002BB8
:1017F00001DD017008BD054B024A7D21F1E700BF04
:1018000008410008843E0008C04100084C40000820
:10181000007870472DE9F7430D9EBDF828900B9D89
:101820009DF83040BDF8388007461946104616B975
:10183000B8F1000F43D11F2C41D83B78D3B9B8F190
:10184000070F39D839F0030339D1424631464FF6F4
:10185000FF70FFF73FFE4FEA092920F0010009F46D
:101860004079400449EA0464400C44EA40244FF6BD
:10187000FF730DE043EA0923B8F1070F43EA04645C
:10188000F5D9FFF701FE42463146FFF723FE034636
:101890008DE840012A4621463846FFF735FE0DB94E
:1018A000FFF750FD2B780133DBB21F2B88BF0023DD
:1018B0002B7003B0BDE8F0836FF00300F9E76FF021
:1018C0000100F6E72DE9F7430E9F0B9D9DF834804C
:1018D000BDF83C6081469DF8300007B9C6BB1F28A3
:1018E00036D899F800E0BEF1000F34D00C0244F075
:1018F00080049DF8281044EAC83444EA014444EACC
:101900000E04072E44EA006415D919461046FFF765
:10191000BBFD32463946FFF7DDFD034601960097D1
:101920002A4621464846FFF7EFFDB8F1010F0CD1DA
:1019300025B9FFF707FD4FF6FF73EFE72B7801336B
:10194000DBB21F2B88BF00232B7003B0BDE8F083F0
:101950006FF00100F9E76FF00300F6E7C06900B12E
:1019600004307047C1690B68C3610C30FFF7F8BCE5
:101970002DE9F84FD0F818A0DFF86C800546164620
:101980001F4654464FF0000900F10C0B0CB9BDE89E
:10199000F88FD4E90223B21A67EB0303994508BF15
:1019A00090451FD2AB699C42214628460DD1FFF7D6
:1019B000EDFCAB691B68AB6121465846FFF7D0FCD4
:1019C000AC692346A2461C46E0E7FFF7DFFC23682C
:1019D000CAF8003021465846FFF7C2FC5446DAF8F0
:1019E0000030EFE72368EDE780841E002DE9F04F1B
:1019F0008BB00D4614460793DDF8509082460028C0
:101A000000F06481B9F1000F00F06081531E3F2B9C
:101A100000F25C81012A03D1079B002B40F0568124
:101A2000BAF81460F6000023B5420893099380F0D9
:101A300053812B199E420AD2761B16F0FF0607D15E
:101A4000AB4BAC4A40F26751AB4802F0BFF82646B8
:101A5000DAF80C3023B9DAF81030002B00F0A5804A
:101A60002F2D31D8C5F1300846454FF000032CBF6B
:101A70005FFA88F8B0460093294608AB4246DAF888
:101A80000800FFF7B7FCA6EB08074544FFB2BAF819
:101A9000143003F10053063BDB000293DAF80C30FC
:101AA00005934FF0300B059B002B51D087B9DAF826
:101AB0001000002861D0002F5FD0AB4550D98F4B6C
:101AC0008C4A40F2A651BFE737464FF00008DEE7E8
:101AD000029B23B98A4B874A4FF4B161B4E7029B5A
:101AE000E02B28BFE02306935B44AB4204931DD94F
:101AF0005B1B9F4226BFDBB203930397AB4504D920
:101B00007E4B7C4A40F291519EE70598CDF80080CB
:101B100008ABA5EB0B01039A0430FFF76BFC039BAA
:101B20009844FF1A1D445FFA88F8FFB2049B9B4556
:101B300004D3744B6F4A40F29B5185E7029B069A8F
:101B4000DDF810B09B1A0293059B1B680593AAE76A
:101B5000029BBB42ABD26C4B664A40F2A15173E789
:101B6000CDF800803A46A5EB0B0108ABFFF742FC2D
:101B7000B8443D445FFA88F80027BAF81430B5EB52
:101B8000C30F04D9614B5B4A40F2B1515CE7B8F135
:101B9000400F04D95E4B574A40F2B25154E767B147
:101BA0005C4B544A40F2B3514EE70093324608ABC7
:101BB0002946DAF80800FFF71DFC731E3F2B35B2EB
:101BC00001D8A64204DD544B544A40F235213BE78C
:101BD00060070AD00AAB03EBD401624211F8083C5B
:101BE00002F00702134101F8083C082C21D9102CFF
:101BF00021D9202C8CBF08230423079A002A6DD0FA
:101C0000B4EBC30F6CD0082C04F1FF3215D89DF84B
:101C1000203023FA02F2D10706D54FF0FF3202FA44
:101C200004F423438DF820309DF8203089F80030EB
:101C30004EE00123E1E70223DFE7102C11D8BDF8C5
:101C4000203023FA02F2D20706D54FF0FF3202FA13
:101C500004F42343ADF82030BDF82030A9F800305B
:101C600036E0202C0ED8089921FA02F2D30705D5C8
:101C70004FF0FF3303FA04F40C430894089BC9F8AF
:101C8000003025E0402C1CD0DDE90867304639469D
:101C9000FEF7A6FA002100F0010050EA01030BD084
:101CA000224601200021FEF7A7FA404261EB4101E4
:101CB00006430F43CDE90867DDE90823C9E900239E
:101CC00006E0174B154A4FF42071BDE66FF0010591
:101CD00028460BB0BDE8F08F1D46F9E7012CA3D0D4
:101CE000082CA1D9102CB7D9202CE5D8C6E700BF05
:101CF000583F0008303F0008C04100087A3F000804
:101D0000673F00089F3F0008C73F0008EE3F0008FC
:101D10001C400008344000084E400008B03E000857
:101D20004C40000830B585B030B9244B244A40F20D
:101D3000B121244801F04AFF23B9234B204A40F245
:101D4000B221F6E7402A04D9204B1D4A40F2B621C1
:101D5000EFE722B91D4B1A4A4FF42F71E9E700242F
:101D6000012A0294039417D11B788DF80830530789
:101D70000AD004AB03EBD203554213F8084C05F02C
:101D80000705AC4003F8084C00910346002102A867
:101D9000FFF730FB05B030BD082AE5D9102A03D87B
:101DA0001B88ADF80830E2E7202A02D81B680293AE
:101DB000DDE7D3E90045CDE90245D8E788400008D2
:101DC000C43E0008C0410008A34000084C40000881
:101DD00070B50C4600F10C05E16819B9A1602161EC
:101DE000A18270BD0E682846FFF7BAFAE660F3E7F5
:101DF0002DE9F04FD1F8009091B0C9F3C016044618
:101E00000D46CDE90223002E50D0C9F3C03BC9F3E3
:101E10000626B9F1000F80F29F8119F0C04F40F003
:101E20009B812B7B002B00F09781BBF1020F03D02D
:101E30002278B24240F0938109F07F02BBF1020F99
:101E4000059236D119F07F0FC9F30F2A01D10AF09C
:101E5000030A2B447606059A93F8038046EA0B465C
:101E600046EA82465FEAD81346EA0A06069300F07D
:101E70009A800022002310A961E90823059B0093A2
:101E800067685B4652462046B847002800F08880C5
:101E9000A7698FB9314604F10C00FFF7DBF907465B
:101EA000D0B96FF0020011B0BDE8F08F4FF0020B17
:101EB000AFE7C9F3074ACCE73B699E420DD03F68C4
:101EC000002FF9D1314604F10C00FFF7C3F90746A2
:101ED0000028E6D0A3693B60A761DDE90801FFF7B0
:101EE000D3FAB882F97D08F01F06C1F38401711A94
:101EF00089B20FFA81FED7E90223BEF1000FB8BF05
:101F000001F1200EC9F30461B8BF0FFA8EFE0791EC
:101F100052EA030100F02F81DDE90201801A61EB32
:101F2000030102460B469F480021994208BF904298
:101F3000C0F02181069B002B3FD0BEF1010F00F3C2
:101F40001A8118F0400F38D0DDE90223C7E90223D7
:101F5000202200210DEB0200FFF706F9DDE9022344
:101F6000CDE908232B1D0A932B7BADF836A0013B4E
:101F7000DBB2ADF834309DF81C308DF83A309DF866
:101F800014308DF83B3020468DF838B08DF839602C
:101F9000A36808A998473846FFF70CFA002082E7A3
:101FA0006FF00B007FE7A76917B96FF00C007AE7B5
:101FB0003B699E4296D03F68F6E7FB7DC8F340122E
:101FC000B2EBD31F40F0CE80C3F38403B34240F0A2
:101FD000CC8006992B7B4FEA981279B3D2073CD478
:101FE000032B40F2C580DDE90223C7E902232B7BE6
:101FF000AE1D033BDBB23246394604F10C00FFF75D
:1020000029FB002808DA39462046FFF7BFF9384691
:10201000FFF7D0F9032046E7AB883B832A7B033ADE
:10202000D2B2B88A3146FFF755FAFB7DB882DA435F
:10203000C2F3C01262F3C713FB75AFE76AB92E1D76
:10204000013BDBB23246394604F10C00FFF702FBDC
:102050000028D8DB2A7B013AE2E7FA8AC2F30902B8
:10206000013B052AD9B250D8281D002399420AD92C
:1020700007EB020E013210F801CB8EF81AC00133C3
:10208000062ADBB2F2D1DDE902898B4207F11A029E
:10209000CDE908890A9238BF04337A680B9234BFBD
:1020A0005B1900230C93FB8AADF836A0C3F3090338
:1020B00019449DF81C308DF83A309DF814308DF895
:1020C0003B300023ADF834108DF838B08DF839600E
:1020D0007B602A7BB88A013A291DFFF7FBF93B8B0D
:1020E000B882834203D1A36808A92046984708A96B
:1020F0002046FFF76DFE3846FFF75CF9B88A3B8B48
:10210000984214BF11200020CDE6786810B34FF03C
:10211000060E03689BB9A2EB0E021B2A13D80332EA
:10212000024405F1040E1F309942ACD91EF801CBD0
:1021300002F801CF01339042DBB2F5D1A3E70EF1F3
:102140001C0E1846E5E7184B184A194840F2B3111F
:1021500001F03CFD034696E76FF00900A3E66FF03F
:102160000A00A0E66FF00D009DE66FF00E009AE603
:102170006FF00F0097E6FB7D68F386036FF3C713DC
:10218000FB7539462046FFF701F9069B002B7FF4CB
:10219000D8AEFB7DC3F38402013262F38603FB7584
:1021A00003E700BF80841E00B84000089C3E000882
:1021B000C0410008026843681143016003B1184739
:1021C000704700002DE9F041504EB04240F0898048
:1021D0004F4CDFF840E1256C45F000752564256E15
:1021E00045F000752566246E446DD4F8007207EA48
:1021F0000E0747F00107C4F80072D4F8005205EA50
:102200000E0545F0010545EA0121C4F80012002A37
:1022100069D00021C4F81C120F46C4F80412C4F897
:102220000C12C4F8141204EBC10501311C29C5F8C5
:102230004072C5F84472F6D14FF0000E4FF0010C19
:10224000964514D1426DD2F80032B04223F001031A
:10225000C2F8003257D12E4B1A6C22F000721A6469
:102260001A6E22F000721A661B6EBDE8F0819F782C
:102270001D8817F0010F18BFD4F804820CFA05F17D
:102280001CBF41EA0808C4F8048217F0020F1EBF01
:10229000D4F80C8241EA0808C4F80C827F0742BFD8
:1022A000D4F814720F43C4F8147204EBC5055F68C8
:1022B000C5F840729F68C5F84472D4F81C5229438F
:1022C000C4F81C120C330EF1010EB9E7446D002165
:1022D000C4F81C12C4F80412C4F80C12C4F8141286
:1022E000AAE7002AF2D1436D0022C3F84022C3F8C6
:1022F0004422C3F80422C3F814220122C3F80C229A
:10230000C3F81C229EE7BDE8F08100BFB83600206C
:10231000003802400000FFFF184B5A6D936810B55B
:1023200013F00104936005D013F00C0F14BF4FF4A9
:1023300080340124D90506D513F4406F14BF44F44A
:10234000003444F00204DA0306D513F4402F14BF1E
:1023500044F4802444F00404202383F311880021F2
:10236000074800F011FE21460648FFF723FF00232F
:1023700083F31188BDE8104001F0B6B8B8360020EC
:10238000C0360020DC36002038B5154C636DDD68A2
:10239000AA0713D05A6922F002025A61202383F35C
:1023A0001188002104F1100000F0EEFD012104F17C
:1023B0001800FFF7FFFE002383F31188EB060BD50F
:1023C000636D1021D960202383F311880548FFF73E
:1023D000F1FE002383F31188BDE8384001F084B892
:1023E000B8360020E836002038B5154C636D1D69FD
:1023F000AA0713D05A6922F010025A61202383F3EE
:102400001188002104F1100000F0BEFD022104F14A
:102410001800FFF7CFFE002383F31188EB060BD5DE
:10242000636D10211961202383F311880548FFF79C
:10243000C1FE002383F31188BDE8384001F054B891
:10244000B8360020E836002038B5144C636D5D685E
:102450005D602A0710D52046032200F8482B1A6831
:1024600022F002021A60202383F311880021FFF773
:10247000A1FE002383F311886B070BD5636D996967
:10248000202383F3118806480904FFF793FE0023F5
:1024900083F31188BDE8384001F026B8B836002033
:1024A000E836002010B50F4C204600F005FA0E4B20
:1024B00063650B21132000F0E7F90B21142000F0D5
:1024C000E3F90B21152000F0DFF90B21162000F0B5
:1024D000DBF9002320461A460E21BDE81040FFF725
:1024E00071BE00BFB836002000640040114B984216
:1024F00010B5044609D1104B1A6C42F000721A64F0
:102500001A6E42F000721A661B6E636D01221A6029
:10251000636D5A68D20707D5626851681268D9613D
:102520001A60064A5A6110BD0121082000F060FCC3
:10253000EEE700BFB8360020003802405B8701009C
:1025400003291AD8DFE801F0020A0F14436D9B68D3
:1025500013F0E05F14BF012000207047436D9868BE
:10256000C0F380607047436D9868C0F3C0607047E7
:10257000436D9868C0F300707047002070470000FA
:1025800010B503291FD8DFE801F0021F2327416D92
:102590008B68C3F30163183301EB031310788106D2
:1025A0001ED55468C0F30011490041EAC40141F04E
:1025B000040100F00F00586090689860D268DA60FB
:1025C00041F00101196010BD436D03F5C073E5E7EB
:1025D000436D03F5C873E1E7436D03F5D073DDE7A1
:1025E0009488C0F30011490041EA4451E1E700003A
:1025F00001290CD003D3022910D000207047436D6D
:10260000DA68920701D1186903E001207047436D31
:10261000D86810F0030018BF01207047436DF2E73F
:1026200010B539B9436DD96889071BD11B699B0760
:1026300004D110BD012915D0022948D1416DD1F82E
:10264000C031D1F8C401D1F8C8411461D1F8CC41EE
:10265000546120240C610C69A40717D14C6944F023
:10266000100412E0416DD1F8B031D1F8B401D1F8C5
:10267000B8411461D1F8BC4154612024CC60CC68CD
:10268000A40703D14C6944F002044C6111795C0841
:1026900064F304119C0864F34511117189064BBF62
:1026A00091681189DB085B0D4CBF63F31C0163F378
:1026B0000A01137948BF916060F3030313714FEA75
:1026C00010234FEA104058BF11811370508010BD85
:1026D000002304491A465A50C8180833802B426018
:1026E000F9D1704710370020026843681143016038
:1026F00003B1184770470000024AD36843F0C00393
:10270000D360704700100140024AD36843F0C00311
:10271000D3607047004400402DE9F041D0F85C647C
:10272000F7683368DA0505469CB20DD5202383F39C
:1027300011884FF400710430FFF7D6FF6FF48073F7
:102740003360002383F31188202383F3118805F17C
:10275000040814F02F0333D183F31188380615D5FC
:10276000210613D5202383F3118805F1380000F0EA
:1027700031FA002846DA0821281DFFF7B5FF4FF689
:102780007F733B40F360002383F311887A060ED5F4
:1027900063060CD5202383F31188EA6C2B6D9A42D3
:1027A00002D12B6C002B2FD1002383F31188D5F895
:1027B0006424D368002B31D01069BDE8F04118477C
:1027C000230713D014F0080F0CBF00218021E0076D
:1027D00048BF41F02001A20748BF41F04001630714
:1027E00048BF41F480714046FFF77EFFA40673683E
:1027F00005D595F860142846194000F08DFA346824
:10280000A4B2A6E77060BEE727F040073F0410219E
:10281000281D3F0CFFF768FFF760C5E7BDE8F081B2
:1028200008B50348FFF778FFBDE8084000F05CBE3C
:102830009037002008B50348FFF76EFFBDE8084059
:1028400000F052BEF83B002010B5094C094A204662
:10285000002100F03FFA084BC4F85C34074C084AEA
:102860000021204600F036FA064BC4F85C3410BD57
:1028700090370020F926000800100140F83B0020A6
:10288000092700080044004000F1604300F01F02E7
:10289000400903F5614309018000C9B200F16040BD
:1028A00083F8001300F5614001239340C0F88031A4
:1028B00003607047FFF7F6BD00F1080201230370C3
:1028C00082600023C26000F11002836143604362B2
:1028D000026103634261C363C36103628362C362D3
:1028E00043638363036443648364C3640365704721
:1028F00010B52023044683F311880223037041603E
:10290000FFF7F4FD03232370002383F3118810BD28
:102910002DE9F0411F4604460D461646202383F359
:10292000118800F108082378042B0ED02946204690
:10293000FFF706FE48B1204632462946FFF720FE43
:10294000002080F31188BDE8F0813946404600F050
:10295000FFFA0028E7D0002383F31188BDE8F08157
:102960002DE9F0411F4604460D461646202383F309
:10297000118800F110082378042B0ED02946204638
:10298000FFF736FE48B1204632462946FFF748FE9B
:10299000002080F31188BDE8F0813946404600F000
:1029A000D7FA0028E7D0002383F31188BDE8F0812F
:1029B000F8B5154682680669AA420B46816938BF98
:1029C0008568761AB542044607D218462A46FEF7AD
:1029D000B9FBA3692B44A3610DE011D93246184617
:1029E000FEF7B0FBAF1B3A46E1683044FEF7AAFBA6
:1029F000E2683A44A261A3685B1BA3602846F8BD65
:102A000018462A46FEF79EFBE368E4E783682DE953
:102A1000F041044693421546266938BF85684069EF
:102A2000361AB5420F4606D22A46FEF78BFB63697B
:102A30002B4463610DE012D93246A5EB0608FEF780
:102A400081FB4246B919E068FEF77CFBE26842442C
:102A50006261A3685B1BA3602846BDE8F0812A463B
:102A6000FEF770FBE368E4E710B50A440024C36195
:102A7000029B006040608460C160816141610261CD
:102A8000036210BD08B582694369934201D182682F
:102A900082B98268013282605A1C426119704269AF
:102AA00003699A4201D3C3684361002100F060FAD0
:102AB000002008BD4FF0FF3008BD000070B5202396
:102AC00004460E4683F31188A568A5B1A368A269E0
:102AD000013BA360531CA36115782269934224BF74
:102AE000E368A361E3690BB120469847002383F3B1
:102AF0001188284670BD3146204600F029FA00288A
:102B0000E2DA85F3118870BD2DE9F74F05460F46CF
:102B100090469A46D0F81C90202686F311884FF0F4
:102B2000000B144664B1224639462846FFF740FFA1
:102B3000034668B95146284600F00AFA0028F1D049
:102B4000002383F31188A8EB040003B0BDE8F08FE5
:102B5000B9F1000F03D001902846C847019B8BF3C1
:102B60001188E41A1F4486F31188DBE7C160816194
:102B70004161C3611144009B00604060826001615B
:102B800003627047F8B504460E461746202383F3C8
:102B90001188A568A5B1A368013BA36063695A1CAD
:102BA00062611E70236962699A4224BFE3686361AF
:102BB000E3690BB120469847002080F31188F8BDE7
:102BC0003946204600F0C4F90028E2DA85F311887E
:102BD000F8BD0000836942699A4210B501D182684C
:102BE0007AB98268013282605A1C82611C7803695A
:102BF0009A4201D3C3688361002100F0B9F92046ED
:102C000010BD4FF0FF3010BD2DE9F74F05460F46C0
:102C100090469A46D0F81C90202686F311884FF0F3
:102C2000000B144664B1224639462846FFF7EEFEF3
:102C3000034668B95146284600F08AF90028F1D0C9
:102C4000002383F31188A8EB040003B0BDE8F08FE4
:102C5000B9F1000F03D001902846C847019B8BF3C0
:102C60001188E41A1F4486F31188DBE70268436881
:102C70001143016003B11847704700001430FFF79B
:102C800043BF00004FF0FF331430FFF73DBF00009B
:102C90003830FFF7B9BF00004FF0FF333830FFF78F
:102CA000B3BF00001430FFF709BF00004FF0FF3141
:102CB0001430FFF703BF00003830FFF763BF000098
:102CC0004FF0FF323830FFF75DBF00000020704743
:102CD000FFF7BABD37B50F4B036000234360836035
:102CE000C360012304460374154600900B464FF45D
:102CF000007200F15C011430FFF7B6FE00942B4621
:102D00004FF4007204F5177104F13800FFF72EFF3D
:102D100003B030BDFC41000838B5C36904460D4618
:102D20001BB904210844FFF7A1FF294604F1140050
:102D3000FFF7A8FE002806DA201D4FF48061BDE8E9
:102D40003840FFF793BF38BD024B00221B605B6029
:102D50009A60704760400020002303748268054B2E
:102D60001B6899689142FBD25A6803604260106008
:102D7000586070476040002008B5202383F3118815
:102D8000037C032B05D0042B0DD02BB983F31188C2
:102D900008BD436900221A604FF0FF334361FFF71B
:102DA000DBFF0023F2E790E80C001A600268536032
:102DB000F2E70000002303748268054B1B689968E2
:102DC0009142FBD85A6803604260106058607047B7
:102DD00060400020054B19690874186802681A6081
:102DE0005360186101230374FDF7A6BA6040002008
:102DF00030B54B1C87B005460A4C10D023690A4AEF
:102E000001A800F0DDF82846FFF7E4FF049B13B1AA
:102E100001A800F011F92369586907B030BDFFF728
:102E2000D9FFF8E760400020792D000838B50C4D37
:102E300041612B6981689A689142044603D8BDE8D4
:102E40003840FFF789BF1846FFF786FF01232C6142
:102E5000014623742046BDE83840FDF76DBA00BF37
:102E600060400020044B1A681B6990689B68984278
:102E700094BF0020012070476040002010B5084C2E
:102E8000236820691A6822605460012223611A7441
:102E9000FFF790FF01462069BDE81040FDF74CBAEE
:102EA0006040002008B5FFF7DDFF18B1BDE808401D
:102EB000FFF7E4BF08BD0000826002220274002216
:102EC000427470478368A3F17C0243F80C2C0269BA
:102ED00043F83C2C426943F8382C074A43F81C2C31
:102EE000C26843F8102C022203F8082C002203F8D1
:102EF000072CA3F1180070475103000810B52023D8
:102F000083F31188FFF7DEFF00210446FFF78EFFF1
:102F1000002383F31188204610BD0000024B1B697B
:102F200058610F20FFF756BF60400020202383F335
:102F30001188FFF7F3BF000008B50146202383F393
:102F400011880820FFF754FF002383F3118808BD80
:102F500049B1064B42681B6918605A6013604360B0
:102F60000420FFF745BF4FF0FF307047604000205E
:102F70000368984206D01A6802605060596118468A
:102F8000FFF7EABE7047000038B504460D462068DA
:102F9000844200D138BD036823605C604561FFF75F
:102FA000DBFEF4E7054B03F114025A619A614FF01E
:102FB000FF32DA6100221A62704700BF60400020D1
:102FC000F8B503614FF08043C2605C6A194B1A4642
:102FD000022952F8145F38BF0221954206461F4667
:102FE0000AD1586198611C620560456081600819CA
:102FF000BDE8F84000F0C6BA186AAB68241A0C198C
:1030000002D3E41A2D6804E09C4202D2204400F06E
:10301000C7FAAB689C42F4D86B68736035601E6079
:103020006E60B460A9684FF0FF33091BA960FB61B3
:10303000F8BD00BF6040002010B41B4C234653F87D
:10304000141F814210D0416802680A600268516012
:103050009A424FF00001C16003D0936881680B442D
:1030600093605DF8044B70470A68626100209A42E1
:103070005360C86003D15DF8044B00F08BBA9368CD
:103080008868034493604FF08042206A526A121AA3
:103090009342E6D9991A012998BF931C18445DF808
:1030A000044B00F07DBA00BF604000200020704754
:1030B000FEE70000704700004FF0FF30704700004F
:1030C000BFF34F8F024AD368DB03FCD4704700BFC5
:1030D000003C024008B5094B1B7873B9FFF7F0FFBD
:1030E000074B1A69002ABFBF064A5A6002F18832AC
:1030F0005A601A6822F480621A6008BDA04000205D
:10310000003C02402301674508B50B4B1B7893B97F
:10311000FFF7D6FF094B1A6942F000421A611A689C
:1031200042F480521A601A6822F480521A601A68B7
:1031300042F480621A6008BDA0400020003C0240BA
:10314000072870B513D80B4A0B4C137863B90B4E94
:103150004FF0006144F8231056F823500133082B38
:103160002944F7D10123137054F8200070BD0020CA
:1031700070BD00BFC4400020A440002024420008CD
:10318000014B53F820007047244200080820704784
:10319000072810B5044601D9002010BDFFF7D0FF65
:1031A000064B53F824301844C21A0BB9012010BD45
:1031B00012680132F0D1043BF6E700BF2442000858
:1031C000072810B5044621D8FFF77AFFFFF782FFE2
:1031D0000F4AF323D360C300DBB243F4007343F020
:1031E00002031361136943F480331361FFF768FF2F
:1031F000FFF7A6FF074B53F8241000F029F9FFF75B
:1032000083FF2046BDE81040FFF7C2BF002010BD7D
:10321000003C0240244200082DE9F84312F001036B
:10322000154640D184182E4A94423CD82D4B1B6839
:1032300013F0010337D02C4CFFF74CFFF323E3606E
:10324000FFF73EFF40F20127032D01D9830713D07A
:10325000254C0F46401A40F20118EB1B0B44012B82
:1032600000EB0706236924D823F001032361FFF74D
:103270004BFF0120BDE8F883236923F440732361E9
:1032800023693B43236151F8046B0660BFF34F8F02
:10329000FFF716FF03689E4208D0236923F001035D
:1032A0002361FFF731FF0020BDE8F883043D0430BF
:1032B000CAE723F440732361236943EA08032361C7
:1032C000B94637F8023B3380BFF34F8FFFF7F8FE64
:1032D0003688B9F80030B6B2B342BED0DDE700BFE1
:1032E000FFFF070800380240003C0240084908B5CB
:1032F0000B7828B153B9FFF7EDFE01230B7008BD21
:1033000023B1BDE808400870FFF7FEBE08BD00BF4E
:10331000A04000204FF0804330B5586A0B4B1A682C
:1033200082421A460FD90A4B0A49D3E9004514F1E3
:10333000FF3445F10005C3E900450B6803F583033D
:1033400003F637130B60106030BD00BFC84000208B
:10335000D0400020CC40002070B500F0A9F906460E
:10336000FFF7D8FF054BD3E90045241845F10005C8
:10337000304600F0A7F92046294670BDD040002015
:1033800038B500F095F90546FFF7C4FF054B4FF43B
:103390007A74B0FBF4F418680444284600F092F9FB
:1033A000204638BDCC40002010B50244064B0439FD
:1033B000D2B2904200D110BD441C00B253F820009C
:1033C00041F8040FE0B2F4E750280040104B30B54C
:1033D0001C6F240407D41C6F44F400741C671C6F1A
:1033E00044F400441C670B4C236843F4807323604F
:1033F0000244094B0439D2B2904200D130BD441C82
:1034000000B251F8045F43F82050E0B2F4E700BF87
:1034100000380240007000405028004007B50122EB
:1034200001A90020FFF7C0FF019803B05DF804FB7D
:1034300013B50446FFF7F2FFA04206D002A901220D
:1034400041F8044D0020FFF7C1FF02B010BD00009D
:1034500070470000074B45F255521A6002225A602D
:1034600040F6FF729A604CF6CC421A60024B012281
:103470001A70704700300040D9400020034B1B7881
:103480001BB1034B4AF6AA221A607047D9400020AC
:1034900000300040034B1B689B0042BF024B0122DF
:1034A0001A70704774380240D8400020024B4FF029
:1034B00080721A60704700BF74380240014B187860
:1034C000704700BFD8400020064A536823F001032C
:1034D0005360EFF30983683383F30988002383F390
:1034E0001188704730EF00E010B5202383F3118876
:1034F000104B5B6813F4006318D0F1EE103AEFF351
:1035000009844FF0807344F84C3C0B4BDB6844F863
:10351000083CA4F1680383F30988FFF7A3FC18B102
:10352000064B44F8503C10BD054BFAE783F3118875
:1035300010BD00BF00ED00E030EF00E061030008C7
:103540006403000870470000FEE70000084A094BCA
:1035500009498B4204D3094A0021934205D370479D
:1035600052F8040F43F8040BF3E743F8041BF4E7A5
:1035700000440008DC420020DC420020DC42002045
:1035800000F034B94FF08043002258631A610222E0
:10359000DA6070474FF080430022DA607047000025
:1035A0004FF0804358637047FEE7000010B5174C9A
:1035B000FFF7CAFBFFF7F6FC802215492046FFF70C
:1035C0007BFC012344F8180C0374124B124AD9688F
:1035D00021F4E0610904090C0A431049DA60CA6861
:1035E00042F08072CA600E490A6842F001020A6025
:1035F0001022DA77202283F82220002383F3118817
:1036000062B60848BDE81040FFF778BC884000204B
:103610004442000800ED00E00003FA05F0ED00E090
:10362000001000E04C4200082DE9F84F1F4C4FF00D
:103630000008656904F11407C1464FF08043266A0B
:103640005B6AAA689E1B96421DD34FF0200AAA68A7
:10365000236AD5F80CB0134423622B68BB425F6029
:10366000A6EB02066361C5F80C8001D1FFF792FF5B
:1036700089F311882869D8478AF311886569AB688E
:103680009E42E4D2D9E76269BA420CD091682362C3
:103690008E1B9660A86802282CBF1818981CBDE8DD
:1036A000F84FFFF77DBFBDE8F88F00BF60400020F6
:1036B000EFF3118020B9EFF30583202282F3118804
:1036C0007047000010B558B9EFF30584C4F308043F
:1036D00014B180F3118810BDFFF7E4FB84F3118867
:1036E00010BD00004B6843608B688360CB68C3608B
:1036F0000B6943614B6903628B6943620B6803602A
:103700007047000008B51F4B1F481A6942F0FF02BE
:103710001A611A6922F0FF021A611A691A6B42F0E3
:10372000FF021A631A6D42F0FF021A65174A1B6DF9
:103730001146FFF7D7FF164802F11C01FFF7D2FF31
:10374000144802F13801FFF7CDFF134802F154018C
:10375000FFF7C8FF114802F17001FFF7C3FF1048DF
:1037600002F18C01FFF7BEFF0E4802F1A801FFF73E
:10377000B9FF0D4802F1C401FFF7B4FFBDE80840EE
:1037800000F09CB800380240000002406C42000883
:103790000004024000080240000C024000100240F9
:1037A0000014024000180240001C024008B500F05E
:1037B000FDF9FFF7FBFEBDE80840FFF76BBE000018
:1037C000704700004FF0804310B51A69920708D582
:1037D00000241C61202383F31188FFF725FF84F365
:1037E0001188BDE81040FFF77FBE0000104B1A6C37
:1037F00042F001021A641A6E42F001021A660D4A82
:103800001B6E936843F0010393604FF080435F2287
:103810009A624FF0FF32DA6200229A615A63DA60EC
:103820005A6001225A6108211A601C20FFF72CB847
:1038300000380240002004E01E4B1A6962F0FF02CB
:103840001A611A69D2B21A614FF0FF301A695A69C7
:10385000586100215A6959615A691A6A62F08052A6
:103860001A621A6A02F080521A621A6A5A6A586216
:103870005A6A59625A6A1A6C42F080521A641A6E75
:1038800042F080521A661A6E0B4A106840F480703B
:103890001060186F00F44070B0F5007F1EBF4FF449
:1038A000803018671967536823F40073536000F081
:1038B0005DB900BF0038024000700040334B344A0D
:1038C0001A64344A4FF4404111601A6842F0010210
:1038D0001A601A689207FCD59A6822F003029A606F
:1038E0002A4B19469A6812F00C02FBD1186800F0B6
:1038F000F90018609A601A6842F480321A600B6806
:103900009B03FCD54B6F43F001034B671F4B5A6F72
:103910009007FCD5204A5A601A6842F080721A60FB
:103920001C4A53685904FCD5184B1A689201FCD5FF
:103930001A4A9A600322C3F88C200022C3F894200C
:10394000174B1A68174B9A42174B1BD1174A11682D
:10395000174A914216D140F203121A600B4B9A6833
:1039600042F002029A609A6802F00C02082AFAD128
:103970005A6C42F480425A645A6E42F480425A664B
:103980005B6E704740F20372E7E700BF0038024009
:10399000000400100070004010604108009088385A
:1039A000002004E011640020003C024000ED00E033
:1039B00041C20F41084A08B5536911680B4003F032
:1039C0000103536123B1054A13680BB1506898474E
:1039D000BDE80840FFF788BD003C014010370020DB
:1039E000084A08B5536911680B4003F0020353619C
:1039F00023B1054A93680BB1D0689847BDE80840E9
:103A0000FFF772BD003C014010370020084A08B59E
:103A1000536911680B4003F00403536123B1054A55
:103A200013690BB150699847BDE80840FFF75CBDCA
:103A3000003C014010370020084A08B5536911685E
:103A40000B4003F00803536123B1054A93690BB19E
:103A5000D0699847BDE80840FFF746BD003C0140EB
:103A600010370020084A08B5536911680B4003F06D
:103A70001003536123B1054A136A0BB1506A98478A
:103A8000BDE80840FFF730BD003C01401037002082
:103A9000174B10B55C691A68144004F478725A61C7
:103AA000A30604D5134A936A0BB1D06A98476006FF
:103AB00004D5104A136B0BB1506B9847210604D5FF
:103AC0000C4A936B0BB1D06B9847E20504D5094AB9
:103AD000136C0BB1506C9847A30504D5054A936C41
:103AE0000BB1D06C9847BDE81040FFF7FDBC00BF9C
:103AF000003C0140103700201A4B10B55C691A6871
:103B0000144004F47C425A61620504D5164A136DD0
:103B10000BB1506D9847230504D5134A936D0BB133
:103B2000D06D9847E00404D50F4A136E0BB1506E68
:103B30009847A10404D50C4A936E0BB1D06E9847F8
:103B4000620404D5084A136F0BB1506F98472304E1
:103B500004D5054A936F0BB1D06F9847BDE810406C
:103B6000FFF7C2BC003C014010370020062108B519
:103B70000846FEF789FE06210720FEF785FE06218E
:103B80000820FEF781FE06210920FEF77DFE0621B2
:103B90000A20FEF779FE06211720FEF775FE0621A2
:103BA0002820BDE80840FEF76FBE000008B5FFF70B
:103BB00043FEFEF78DFDFEF77DFEFFF789F8FFF768
:103BC000FFFDBDE80840FFF7DBBC00001FB51C4649
:103BD000094B1B680546D86852B1084B02928DE824
:103BE0000A0022462B460649FDF7CAFA00F042F8C1
:103BF000044B1A46F2E700BF182500204C4300088A
:103C000059430008873D000810B50139024490422D
:103C100001D1002010BD10F8013B11F8014FA34263
:103C2000F5D0181B10BD00002DE9F8430746884663
:103C300091461E468BB10D46A8EB0500B54207EB39
:103C4000000402D20020BDE8F883324649462046EF
:103C5000FFF7DAFF18B1013DEEE7BDE8F883204633
:103C6000BDE8F883034611F8012B03F8012B002A65
:103C7000F9D1704708B5062000F02CF80120FFF7B5
:103C800017FA00001F2938B504460D4604D916233B
:103C900003604FF0FF3038BD426C12B152F8213052
:103CA0004BB9204600F030F82A4601462046BDE8D0
:103CB000384000F017B8012B0AD0591C03D1162345
:103CC0000360012038BD002442F82540284698476B
:103CD000002038BD024B01461868FFF7D3BF00BF74
:103CE0001825002038B5074C002305460846114624
:103CF0002360FFF7E1F9431C02D1236803B12B6075
:103D000038BD00BFD8420020FFF7D0B940A2E4F18F
:103D1000646891064E6F20617070207369670A00B5
:103D2000426164206677206C656E67746820257533
:103D30000A0042616420626F6172645F69642025D9
:103D4000752073686F756C642062652025750A00A4
:103D500042616420617070204352432030782530E6
:103D600038783A30782530387820307825303878EF
:103D70003A3078253038780A00476F6F64206669DA
:103D8000726D776172650A00726563656976656454
:103D90005F756E697175655F69645F6C656E203C07
:103DA0002055415643414E5F50524F544F434F4C64
:103DB0005F44594E414D49435F4E4F44455F49442E
:103DC0005F414C4C4F434154494F4E5F554E495112
:103DD00055455F49445F4D41585F4C454E475448F7
:103DE000002E2E2F2E2E2F546F6F6C732F41505F8D
:103DF000426F6F746C6F616465722F63616E2E63C6
:103E0000707000616C6C6F63617465645F6E6F6489
:103E1000655F6964203C3D20313237006F72672E48
:103E20006172647570696C6F742E637561765F671B
:103E300070730000766F69642068616E646C655F02
:103E4000616C6C6F636174696F6E5F726573706FC4
:103E50006E73652843616E617264496E7374616E3E
:103E600063652A2C2043616E6172645278547261DA
:103E70006E736665722A290063616E617264496EB1
:103E80006974000063616E6172645365744C6F63A2
:103E9000616C4E6F646549440000000063616E61AF
:103EA000726448616E646C6552784672616D65003B
:103EB00063616E6172644465636F64655363616CD2
:103EC0006172000063616E617264456E636F646568
:103ED0005363616C61720000696E6372656D656E3B
:103EE000745472616E73666572494400656E7175D3
:103EF00065756554784672616D6573007075736899
:103F000054785175657565007072657061726546AB
:103F10006F724E6578745472616E736665720000DC
:103F2000636F7079426974417272617900000000B8
:103F30006465736361747465725472616E736665EF
:103F4000725061796C6F6164000000006672656593
:103F5000426C6F636B0000006269745F6C656E6732
:103F60007468203E20300072656D61696E696E670D
:103F70005F62697473203E203000696E7075745FF3
:103F80006269745F6F6666736574203E3D20626C83
:103F90006F636B5F6269745F6F66667365740062FE
:103FA0006C6F636B5F656E645F6269745F6F66669A
:103FB000736574203E20626C6F636B5F6269745F2F
:103FC0006F66667365740072656D61696E696E67B0
:103FD0005F6269745F6C656E677468203C3D207237
:103FE000656D61696E696E675F6269747300696EA1
:103FF0007075745F6269745F6F6666736574203C88
:104000003D207472616E736665722D3E7061796CCD
:104010006F61645F6C656E202A2038006F75747064
:1040200075745F6269745F6F6666736574203C3D8A
:104030002036340072656D61696E696E675F626912
:10404000745F6C656E677468203D3D203000287297
:104050006573756C74203E20302920262620287236
:104060006573756C74203C3D20363429202626204B
:1040700028726573756C74203C3D206269745F6CB6
:10408000656E67746829000064657374696E617495
:10409000696F6E20213D202828766F6964202A29C7
:1040A00030290076616C756520213D202828766FC7
:1040B0006964202A293029006F66667365745F770A
:1040C000697468696E5F626C6F636B203C20283393
:1040D0003255202D205F5F6275696C74696E5F6F69
:1040E00066667365746F66202843616E6172644210
:1040F0007566666572426C6F636B2C2064617461D7
:10410000292900006F75745F696E7320213D202896
:1041100028766F6964202A29302900007372635F52
:104120006C656E203E203055000000002863616EF3
:104130005F6964202620307831464646464646462A
:104140005529203D3D2063616E5F696400000000D9
:10415000616C6C6F6361746F722D3E73746174690E
:1041600073746963732E63757272656E745F7573B1
:104170006167655F626C6F636B73203E2030000087
:104180007472616E736665725F696420213D2028D8
:1041900028766F6964202A293029000073746174BD
:1041A000652D3E6275666665725F626C6F636B73E8
:1041B000203D3D202828766F6964202A2930290077
:1041C0002E2E2F2E2E2F6D6F64756C65732F6C69DC
:1041D0006263616E6172642F63616E6172642E63EB
:1041E000006974656D2D3E6672616D652E64617443
:1041F000615F6C656E203E20300000000000000012
:10420000992C0008852C0008C12C0008AD2C000852
:10421000B92C0008A52C0008912C00087D2C000862
:10422000CD2C0008004000000040000000400000CD
:104230000040000000000100000002000000020039
:10424000000002006D61696E000000006442000819
:10425000E0400020D842002001000000A9350008FD
:104260000000000069646C6500000000A0000028E8
:1042700000000000AAAAAAAA50000000FFFF000048
:10428000007700000000000000A40A010000000008
:10429000AAA6AAAA80500000DFEF00000000007765
:1042A000880000000000000000000000AAAAAAAADE
:1042B00000000000FFFF0000000000000000000000
:1042C0000000000000000000AAAAAAAA0000000046
:1042D000FFFF0000000000000000000000000000E0
:1042E00000000000AAAAAAAA00000000FFFF000028
:1042F00000000000000000000000000000000000BE
:10430000AAAAAAAA00000000FFFF00000000000007
:10431000000000000000000000000000AAAAAAAAF5
:1043200000000000FFFF000000000000000000008F
:1043300000000000000000000A0000000000000073
:104340000300000000000000000000002C20667543
:104350006E6374696F6E3A2000617373657274697D
:104360006F6E2022257322206661696C65643A2095
:1043700066696C6520222573222C206C696E65208D
:104380002564257325730A00FFFFFFFF74000000FA
:104390006400000000000000FE2A0100D2040000BA
:1043A0001C250020000000000000000000000000AC
:1043B00000000000000000000000000000000000FD
:1043C00000000000000000000000000000000000ED
:1043D00000000000000000000000000000000000DD
:1043E00000000000000000000000000000000000CD
:1043F00000000000000000000000000000000000BD
:0444000000000000B8
:00000001FF
